:1030000039C0000063C0000061C000005FC0000064
:103010005DC000005BC0000059C0000057C0000048
:1030200055C0000053C0000051C00000D8C10000CE
:103030004DC000004BC0000049C0000047C0000068
:1030400045C0000043C0000041C000003FC0000078
:103050003DC000003BC0000039C0000037C0000088
:1030600035C0000033C0000031C000002FC0000098
:103070002DC0000011241FBECFEFD2E0DEBFCDBFB8
:1030800004B603FE0EC08091540190915501823424
:103090009C4D39F41092550110925401E0E0F0E09B
:1030A000099511E0A0E0B1E0E2E4F7E302C0059089
:1030B0000D92AA34B107D9F721E0AAE4B1E001C02A
:1030C0001D92A435B207E1F702D039C399CF84B776
:1030D000877F84BF88E10FB6F894809360001092D8
:1030E00060000FBE81E085BF82E085BF69D1789422
:1030F00080910001882311F007D3FACF8091E0007E
:1031000081608093E00082E49CED90935501809370
:1031100054012CE088E190E00FB6F894A8958093D4
:1031200060000FBE20936000FFCF42E361EC81E0BE
:10313000E1C080914C018F77813209F05CC08091B1
:103140004D01893009F057C08091E800877F809356
:10315000E8008091E80082FFFCCF3091F1002091DF
:10316000F100832F922F8F3F2FEF920719F41092C7
:1031700000013BC023E0FC0120935700E89507B60F
:1031800000FCFDCF20E030E061E04091F2004423FC
:10319000D9F0E091F1007091F1004E2F572FF90115
:1031A000EE0FFF1FE80FF91F0A0160935700E89523
:1031B00011242F5F3F4F2034310539F725E0FC0102
:1031C00020935700E8950AC04091E8004B77409360
:1031D000E8004091E80042FFFCCFDBCF07B600FCDF
:1031E000FDCF81E180935700E8958091E8008B77CF
:1031F0008093E80093C00895913049F0923061F0D7
:10320000913279F489E090E023E131E00EC082E16F
:1032100090E023E231E009C082E290E021E031E079
:1032200004C085E190E025E331E0FA013183208399
:10323000089520915201309153012617370748F025
:103240006115710539F42091E8002E772093E8008C
:1032500001C0B90120E061157105C9F13EB3332306
:1032600009F442C0353009F441C03091E80033FD23
:103270003FC03091E80032FF06C08091E80082FF35
:1032800029C080E008953091E80030FFE4CF20911C
:10329000F20030E0FC01281B390BCF01820F931F95
:1032A0006115710549F08830910530F48191809362
:1032B000F10061507109F1CF21E0089709F020E099
:1032C0008091E8008E778093E800CF01C4CF211170
:1032D000C5CFD3CF8EB3882339F0853039F08091B4
:1032E000E80083FFCACF04C082E0089583E0089518
:1032F00081E008958F708093E900EBEEF0E080812B
:1033000081608083EDEEF0E010826093EC004083FA
:103310008091EE00881F8827881F089580914C01B6
:1033200087FD05C08091E80080FF0DC010C080912E
:10333000E80082FD04C08EB38111F9CF0895809119
:10334000E8008B7707C08EB38111ECCF0895809190
:10335000E8008E778093E80008953BD03DD08091BF
:10336000D8008F778093D8008091D80080688093B0
:10337000D8008091D8008F7D8093D80019BC82E05E
:1033800089BD09B400FEFDCF1EBA10924A0142E089
:1033900060E080E0AFDF8091E1008E7F8093E1000C
:1033A0008091E20081608093E2008091E200886079
:1033B0008093E2008091E0008E7F8093E00008958A
:1033C000E3E6F0E080818E7F808381E080934B0193
:1033D000C4CF1092E20008951092E10008951F9268
:1033E0000F920FB60F9211242F933F934F935F9339
:1033F0006F937F938F939F93AF93BF93EF93FF93BD
:103400008091E10080FF16C08091E20080FF12C031
:103410008091E2008E7F8093E2008091E2008061E3
:103420008093E2008091D80080628093D80019BC1C
:103430001EBA69D18091E10084FF2DC08091E20025
:1034400084FF29C019BC82E089BD09B400FEFDCF0C
:103450008091D8008F7D8093D8008091E1008F7E8D
:103460008093E1008091E2008F7E8093E200809162
:10347000E20081608093E20080914A01882311F08C
:1034800084E007C08091E30087FF02C083E001C0B1
:1034900081E08EBB38D18091E10083FF21C0809113
:1034A000E20083FF1DC08091E100877F8093E100EF
:1034B00082E08EBB10924A018091E1008E7F809362
:1034C000E1008091E2008E7F8093E2008091E20033
:1034D00080618093E20042E060E080E00BDF13D186
:1034E000FF91EF91BF91AF919F918F917F916F91DC
:1034F0005F914F913F912F910F900FBE0F901F90B2
:1035000018951F93CF93DF9300D0CDB7DEB7ECE4CF
:10351000F1E08091F100819381E0E435F807C9F78B
:1035200008DE8091E80083FFDAC090914C01809121
:103530004D01853009F465C030F4813059F168F0EF
:10354000833041F1CCC0883009F49CC0893009F443
:10355000ABC0863009F0C3C075C0903881F0923896
:1035600009F0BDC0809150018F708093E900909167
:10357000EB0095FB992790F91092E90001C090E0CB
:103580008091E800877F8093E8009093F10010928B
:10359000F10083C0292F2D7F09F0A1C0923009F0DE
:1035A0009EC090914E01911126C0209150012F7024
:1035B00009F495C02093E9009091EB0090FF1BC0A7
:1035C000833021F48091EB00806213C08091EB0086
:1035D00080618093EB0081E090E0022E01C0880FB3
:1035E0000A94EAF78093EA001092EA008091EB00D7
:1035F00088608093EB001092E9008091E800877F5B
:103600004FC091116CC010914E011F778091E30063
:103610008078812B8093E3008091E800877F8093FE
:10362000E8007CDE8091E80080FFFCCF8091E30021
:1036300080688093E300112311F083E001C082E0F1
:103640008EBB4DC09058923008F049C0AE014F5F1C
:103650005F4F6091500180914E0190914F01CCDD00
:10366000009709F43CC02091E800277F2093E800F0
:10367000BC0189819A81DDDD8091E8008B778093A0
:10368000E8002DC0903859F58091E800877F80933D
:10369000E80080914A018093F1008091E8008E77E4
:1036A0008093E8003BDE1BC0911119C090914E0140
:1036B0009230A8F48091E800877F8093E80090938F
:1036C0004A012CDE80914A01811104C08091E300FF
:1036D00087FF02C084E001C081E08EBB26DD8091BF
:1036E000E80083FF0AC08091E800877F8093E800AC
:1036F0008091EB0080628093EB000F900F90DF9140
:10370000CF911F9108950895CF938EB38823A9F088
:103710008091E9008F709091EC0090FF02C090E8DA
:1037200001C090E0C92FC82B1092E9008091E800F9
:1037300083FDE7DECF70C093E900CF910895F89440
:02374000FFCFB9
:103742000109022200010100803209040000010384
:103752000000000921110100012215000705810363
:103762004000051201100100000008EB0367200170
:10377200000000000106DCFF09FBA101090215009F
:0A37820025FF75089682009102C031
:0400000300003000C9
:00000001FF
